:020000040000FA
:040000002C214E2938
:08000800F000030EF100831269
:10001000031383130408F2000A08F3008C18192054
:1000200073088A0072088400710E8300F00E700E4F
:1000300009008C104E0895004F0893002208A6076F
:1000400023080318230FA70724080318240FA80761
:1000500025080318250FA9078B20AA00A620AA1B94
:100060005628A1012E08AA0C0318A107A10CAA0C5E
:100070000318A107A10CAA0C0318A107A10CAA0C34
:100080000318A107A10CAA0C0318A107A10CAA0C24
:100090000318A107A10CAA0C0318A107A10CAA0C14
:1000A0000318A107A10C8030A1077F28A1012A080D
:1000B000A102AA012E08A10C0318AA07AA0CA10CE0
:1000C0000318AA07AA0CA10C0318AA07AA0CA10CD2
:1000D0000318AA07AA0CA10C0318AA07AA0CA10CC2
:1000E0000318AA07AA0CA10C0318AA07AA0CA10CB2
:1000F0000318AA07AA0C8030A1002A08A102CE1278
:100100004E1221184E16A118CE160310210CCF0046
:100110000310CF0C080007308A0029088200023043
:100120008A00AB30AB002F3084001030CD00A4200B
:100130008000AB0A03198A0A840ACD0B9728AE0106
:10014000AD01AC01AB0108002B088200A019B72853
:10015000201AD628A01A0A29201B0F29AF28201CF4
:100160000800AE01AD01AC01AB01A015B728201C01
:10017000D3282F0803182F0FAB0730080318300FB0
:10018000AC0731080318310FAD0732080318320FDE
:10019000AE07031C0800FF30AB00AC00AD00AE00A2
:1001A000A01120160800A01120170F29201C0729D4
:1001B0003308031C330FAB023408031C340FAC02AA
:1001C0003508031C350FAD023608031C360FAE028E
:1001D000031CFC283708031C370F2B023808031CAC
:1001E000380F2C023908031C390F2D023A08031C62
:1001F0003A0F2E02031808003708AB003808AC008D
:100200003908AD003A08AE002012A01608002012EE
:1002100020170F2920180800A01220170F292018D6
:1002200029293B08031C3B0FAB023C08031C3C0F75
:10023000AC023D08031C3D0FAD023E08031C3E0FFF
:10024000AE0203180800AB01AC01AD01AE012013F2
:1002500008002013A015B7288301F4018500831638
:10026000393085000130950007308100831281010B
:100270000C3095008030930083163F30920083123B
:10028000183092000730990083169F018312403086
:100290008B00831602308C0083120800203084000B
:1002A0001F30FD210C30CE008030CF008F204B144A
:1002B0008B171215811F5A298101AB21A0186321C8
:1002C000740885005A29C90803196829C903080058
:1002D000CA1F7529F8304A0203198D29FF304A02D6
:1002E000031985292010F4108D294A08C000C02167
:1002F0008B134308A2004408A3004508A400460845
:10030000A50020148B17F4148D29201DA729201077
:10031000F4100230C8000530C70048088A009C214C
:10032000C900C70A0319C80A48088A009C21CA00E4
:10033000C70A0319C80A6329470882000230C800A7
:100340000530C700C901F830CA00A0140800201009
:10035000F410A01008002011851D20150508013992
:10036000CD00CB02CB00031D08004D08CC02CC0011
:10037000031908004D08031D0800A01C9E29A72989
:10038000C1014008C20060304202031CC929C200FA
:10039000C11530304202031CCF29C200411518306C
:1003A0004202031CD529C200C1140C304202031CB6
:1003B000DB29C20041144108093CC10006308A0013
:1003C000C20D420DFC39D03ECD00FB21C300CD0A49
:1003D000FB21C400CD0AFB21C500CD0AFB21C600CC
:1003E000C1080319FA290310C60CC50CC40CC30CB0
:1003F000C10BF32908004D088200CD008001840A5A
:06040000CD0BFE290800EF
:04040600003400348A
:06040A0000344F342334DE
:10041000803404344F342334803404344C34233453
:10042000803404344F34233480340434513423343E
:10043000803404344F342334803404344C3447340F
:10044000803408344C342334803404344A34463401
:1004500080342F344C342334803404344A344634CA
:1004600080342F344F342334803404344F342334D5
:10047000803404344C342334803404344F342334F3
:100480008034043451342334803404344F342334DE
:10049000803404344C344734803408344A3446348D
:1004A000803408344C342334803404344A342334C4
:1004B0008034043448344634803456344834463426
:1004C000803408344C342334803404344F3423349F
:1004D00080340434543447348034563451344634F0
:1004E0008034083454342334803404345134233475
:1004F000803404344F344634803456344F342334FB
:10050000803404344F342334803404344C34233462
:10051000803404344F34233480340434513423344D
:10052000803404344F342334803404344C3447341E
:10053000803408344A344634803408344C3423340C
:10054000803404344A342334803404344834463408
:1005500080345634FF34EF348D3421340034EC349D
:100560008D3421340034003400340034E034D83485
:060570001B34433400348B
:100DA0006334EA34DD3436341234213421343A34B5
:100DB000D634013496343D34B43480343F34413435
:100DC000A534BE342034453443340C343D344934E6
:100DD0009F34EC3497344D343F3418343534523426
:100DE0004C34803418345734F334513446345C3442
:100DF000F334F934C23461346734283493346734BB
:100E0000003407340F3417341F3426342E3435346D
:100E10003C34433449344F3454345A345F346334AB
:100E200067346B346E347134743476347834793496
:100E30007A347B347C347C347C347C347C347B3436
:100E40007B347A347A34793478347834773477343C
:100E50007634763475347534753475347534753448
:100E600076347634773477347834793479347A3424
:100E70007B347C347C347D347D347E347E347E34EB
:100E80007E347E347E347E347D347C347C347A34DB
:100E90007934783476347434723470346E346B341C
:100EA00069346634633460345D345A3457345434AE
:100EB00051344E344B3449344634433440343D3459
:100EC0003B3438343534333431342E342C342A34F2
:100ED000283426342434223420341F341D341B3467
:100EE00019341834163415341334113410340E34C4
:100EF0000D340B340934083406340434033401341B
:100F00000034FF34FD34FC34FA34F834F734F5346B
:100F1000F334F234F034EF34ED34EB34EA34E834C3
:100F2000E734E534E334E134E034DE34DC34DA341D
:100F3000D834D634D434D234CF34CD34CB34C8348E
:100F4000C534C334C034BD34BA34B734B534B23424
:100F5000AF34AC34A934A634A334A0349D349A34CD
:100F600097349534923490348E348C348A34883467
:100F700087348634843484348334823482348234B3
:100F800082348234823482348334833484348434AB
:100F900085348634873487348834893489348A3474
:100FA0008A348B348B348B348B348B348B348A344B
:100FB0008A34893489348834883487348634863452
:100FC000853485348434843484348434843485345E
:100FD0008634873488348A348C348F349234953410
:100FE00099349D34A134A634AC34B134B734BD3413
:100FF000C434CB34D234DA34E134E934F134F93462
:084000000000010001000000B6
:02400E00C23FAF
:00000001FF
